:020000020000FC
:1000000004E00EBF0FE50DBF00E00ABD08BD03BD53
:100010000FEF07BB002708BB01EA0FBD01E00EBDD3
:1000200001E605BD06D00BD010D015D01AD01FD0D8
:10003000F9CF43954ABD21D04F3FD9F708954A954E
:100040004ABD1BD04030D9F70895539558BD15D0FF
:100050005F3FD9F708955A9558BD0FD05030D9F762
:100060000895639563BD09D06F3FD9F708956A95E8
:1000700063BD03D06030D9F7089513E426EC2A95C8
:0A008000F1F71A95D9F70000089572
:00000001FF
